:10000000B2011F290408A7008710071007118316E3
:10001000871007100711F030880583122708B218DF
:100020002F283A30A1009830E5203330A600442034
:100030001330A1008830E52044206430E4204420BF
:100040006430E4202230A600442028302E200C30DA
:100050002E2006302E20B21427082F283214A60096
:10006000321C3D280710033C031C42284220073065
:10007000A100D030E520031408003214FE3C03191F
:100080001A290714A60E321C32108714F030880586
:1000900026080F3988048710A60E321844283230FB
:1000A000E420031408000408A60036088400803009
:1000B000B3050830A70003100318B30A6D20A60C7F
:1000C000A70B5C280000AB1A330C6D201D21031414
:1000D0006D202F08A3002E08D8288413AB1F7C287E
:1000E000000834042B1F34068000841700083404F1
:1000F000031C34068000872800083404031C3406DF
:100100002B1B3406800084173409800587282B08B0
:100110001F39FF3EA1002A08F53E0318A10A00007E
:10012000E528B31329080319B3170530A8002730B1
:10013000A3001030A7200330A300E830A720A301BC
:100140006430A720A3010A30A7202408AE28A2000B
:100150002508A1002408A000F9202008A000A80379
:100160000319B31329080319B82828020318080033
:100170002008031DB313B31B0800303E1529A0004F
:10018000A00DA00D200D3839C1389F000030A1000E
:100190001430E5201F151F19CB28A1011E081A29AC
:1001A00083178001840AFF3E031DD1281A29A30169
:1001B000A200FF30A207031CA307031C1A29033067
:1001C000A100DF30E520D928A101E83EA000A10967
:1001D000FC30031CEE28A0070318EB28A0076400DE
:1001E000A10FEB282018F428A01CF8280000F828FC
:1001F0000800A501A4011030A600210DA40DA50D35
:100200002208A4022308031C230FA50203180F29A8
:100210002208A40723080318230FA5070310A00D25
:10022000A10DA60BFD2820081A29840031088A0098
:100230003008820083130313831264000800203007
:10024000840060308A01D120A030840050308A01BF
:10025000D1201030840060308A01D020903084009A
:1002600060308A01D0200130A300F4308A01D82008
:10027000FE308A01032001308A01032083160730F3
:10028000850002309F00861506170516861609148C
:100290008914831200308A01BF20B8003808A000FA
:1002A000A1011930A200A3018A01F920B80064005D
:1002B0008A110A12861D86290730B6004030B40024
:1002C000BC30AA00AB01AE01AF0152308A0154200C
:1002D000A9013808A400A5015330B000B1018A017A
:1002E00091200730B6004030B400BC30AA00AB010A
:1002F000AE01AF014A308A01542020308A015420D7
:1003000020308A01542031308A01542064008A113F
:100310000A12061FB5290730B6004030B400BC30C1
:10032000AA00AB01AE01AF0152308A015420A901ED
:100330003808A400A5015330B000B1018A01912012
:100340000730B6004030B400BC30AA00AB01AE01AB
:10035000AF014A308A01542020308A0154202030D5
:100360008A01542032308A01542064008A110A1212
:10037000051EE4290730B6004030B400BC30AA00A6
:10038000AB01AE01AF0152308A015420A9013808F7
:10039000A400A5015330B000B1018A0191200730BB
:1003A000B6004030B400BC30AA00AB01AE01AF01D2
:1003B0004A308A01542020308A01542020308A019A
:1003C000542033308A01542064008A110A12861E98
:1003D000132A0730B6004030B400BC30AA00AB018D
:1003E000AE01AF0152308A015420A9013808A4009F
:1003F000A5015330B000B1018A0191200730B60049
:100400004030B400BC30AA00AB01AE01AF014A30AD
:100410008A01542020308A01542020308A0154203F
:1004200034308A01542064008A110A12091C422ABD
:100430000730B6004030B400BC30AA00AB01AE01BA
:10044000AF0152308A015420A9013808A400A50147
:100450005330B000B1018A0191200730B60040301E
:10046000B400BC30AA00AB01AE01AF014A308A0132
:10047000542020308A01542020308A015420353005
:100480008A01542064008A110A12891C712A0730DB
:10049000B6004030B400BC30AA00AB01AE01AF01E1
:1004A00052308A015420A9013808A400A501533014
:1004B000B000B1018A0191200730B6004030B4008D
:1004C000BC30AA00AB01AE01AF014A308A01542012
:1004D00020308A01542020308A01542036308A018D
:1004E0005420FE308A01032001308A01032020308D
:1004F0008A01032020308A01032020308A01032052
:1005000020308A01032050308A0103206C308A0198
:10051000032065308A01032078308A010320693086
:100520008A01032020308A01032042308A010320FF
:100530006F308A01032074308A01032020308A0141
:10054000032020308A01032020308A010320FE305E
:100550008A010320C0308A01032053308A0103201E
:1005600070308A01032065308A01032065308A01DA
:10057000032064308A0103203A308A0103202030AE
:100580008A01032020308A01032020308A010320C1
:1005900020308A01032020308A01032020308A0184
:1005A000032020308A0103200230A9003808A4006B
:1005B000A5010230B000B1018A0191208A014A29C7
:0605C00063008A01E02A3D
:02400E007D3FF4
:00000001FF
